:030000000219FDE5
:03000B000200A848
:03002B0002015E71
:03005B000202DDC1
:030073000202C3C3
:1000800002030406080C10182030406080040608A3
:100090000C10182030406080A0C000070F1F3F05E3
:1000A000050D050205030302C2AFC0D0C0E0206207
:1000B00017E5256002E473E525F4F58A758B00D217
:1000C00062D0E0D0D0D2AF3285268AC262E526F473
:1000D0006030758B00D0E0D0D0C295C294C293D26C
:1000E000AF32C295C294C293206E0D20660A740589
:1000F000D5E0FDE57EF45290758B00D0E0D0D0D2F3
:10010000AF32758A00C28DD26201F801B73068053E
:10011000206602D29501B7306805206602D29401AC
:10012000B7306805206602D29301B7D29230680AD0
:100130002066077403D5E0FDD29501B7D2913068EF
:100140000A2066077403D5E0FDD29401B7D290303F
:10015000680A2066077403D5E0FDD29301B7C2AFE9
:10016000C2AD53E6EFC0D0C0E0D2D3D2AFC2CEE52D
:100170002A6007207449152A21BF7800790020746D
:100180002EE580307E01F430E70278FF53DACF208D
:100190007E0343DA20307E0343DA10C2D8C271E511
:1001A00080307E01F430E70279FFC3E89970CB30EC
:1001B0006103752A18207403752A18885FD270208D
:1001C000740DE52B6004152B21CF43DA01C2D82032
:1001D00070024131A85F206102C270207431C3E80F
:1001E00094F0400374F0F8E8C4540F28F87984B709
:1001F0000302410FC313C3138721200802C3132036
:100200000A06C3C898F8410F28F8500374FFF8C3D2
:10021000E895685003E568F88822E52D54066011DA
:10022000E533C313C31324062522F5225003752298
:10023000FF852224A824C3E52495644002A864888D
:1002400025E56970024175C3E8AA699A5003E8FA86
:10025000E4F9EAC333FBE56BF45B29400D256AF84A
:10026000E56A6002156A400B41750AC3E56A9A5057
:1002700002056A78FF8826C3E52594404002D264CF
:1002800020CF0AD0E0D0D043E610D2AD32C2CF05A5
:100290003A7801E52A6005307402152AC3E55F94B7
:1002A00001400575620041B9756300756C00E56237
:1002B0002401F56250037562FFD0E0D0D043E61010
:1002C000D2AD32C2AFC0D053E67FC2607591008517
:1002D0005694855795759104D0D0D2AF32C2AF53A2
:1002E000E6EFC2ADC0D0C0E0C0F0D2D3D2AFA8FB21
:1002F000A9FCC2D8307102614453DACF207E034397
:10030000DA10307E0343DA20D271E580307E01F4CA
:1003100020E702611B88278928A16B53DACF207E52
:100320000343DA20307E0343DA10C2D8C27130743E
:1003300002A1577800E580307E01F430E702A15732
:10034000885FA13F53DACF207E0343DA20307E035B
:1003500043DA10C271206102811D53DACF207E037F
:1003600043DA10307E0343DA20C2D8D271885A892A
:100370005BC3E89558F8E99559F97B007E087A0047
:10038000C3E8948CE994005005755E00810F8821C4
:1003900078A2E6A8216055C3E894C8E99400500803
:1003A000E4D2E4FB7A0A61EAC3E89468E994015074
:1003B00008E4D2E3FB7A0F61EAC3E894D0E994023F
:1003C0005008E4D2E2FB7A1E61EAC3E894A0E99403
:1003D000055008E4D2E1FB7A3C61EAC3E89498E96D
:1003E00094085008E4D2E0FB7A787E00C3E8955C7C
:1003F000FCE9955DFD30E70AECF42401FCEDF434F2
:1004000000FD755E00C3EC9AED9E5003755E018899
:100410005C895D855A58855B597802A13FC3E89590
:1004200027F8E99528F9307C02A123307B02A1232B
:10043000307A02A11C2075028140E9FDE8FC815F51
:10044000E9C313F9E813F8307902A11CE9C313F9E1
:10045000E813F8307802A11CE9C313FDE813FC206F
:100460006126C3EC941CED940240028176ED701875
:0F047000C3EC94C850120529C3E529940A500221
:10047F00A157755F00D270A157E529600215297841
:10048F0088E6F97400207F087896B90302789EE613
:10049F0024FAFEE43400FFC3EC9EFCED9FFD9208AE
:1004AF00B90310A2085007207609D27681C23076A0
:1004BF0002C276A2085016B9030DECF42401FCED2C
:1004CF00F43400FD0204DC78007900A123B9031590
:1004DF00EC33FCED33FDC3EC940AFCED9400FD50BE
:1004EF00047C007D00C3EC94FFED9400400678FF80
:1004FF007900A123EC8575F0A4C5F0A2F733F87944
:10050F0000400302053F78FF790002053FE9C3135E
:10051F00F9E813F8307C0EE9600278FFC3E813386E
:10052F00F8E43400F9C3E894FFE99400400278FF3F
:10053F00885FD270206102A157741FF4552F4BF5BD
:10054F002FC274EB7002D274752A18307403752A97
:10055F000A306102A16B20740353DAFE2074037515
:10056F002B06D0F0D0E0D0D0D2AD43E610327901D7
:10057F0002059B790302059B790A02059B791E02EE
:10058F00059B796402059B79C802059B7817E4D512
:10059F00E0FDD8FAD9F6227A147B780205C27A10D8
:1005AF007B8C0205C27A0D7BB40205C27A0B7BC825
:1005BF000205C27902B27DE4D291D5E0FDD294D585
:1005CF00E0FDC294D5E0FDC291D5E0FDD295E57670
:1005DF00D5E0FDC2957496D5E0FDD9D9EAF8D5E0FE
:1005EF00FDD8FBDBCED29122C37C007D0075F000DD
:1005FF0005F0EA33FAEB33FB50F6EB13FBEA13FA91
:10060F00C3E9FFE8FEE89AF8E99BF95004EFF9EE29
:10061F00F8B3EC33FCED33FDD5F0DFEDF9ECF82258
:10062F00E889F08A20D2D4F8A9F07B0030F70B7B51
:10063F00FFF42401F8E9F43400F9E88520F0A4ADC3
:10064F00F0F8E98520F0A4AFF0FEED2EF974003F2D
:10065F00FA7C04C3EA13FAE913F9E813F8DCF48B14
:10066F00F030F70AE8F42401F8E9F43400F9E889E6
:10067F00F0C2D4F8A9F02222C3E54113F9E54013E3
:10068F00F8C3E54598F8E54699F9500CC3E894800E
:10069F00E994FF40160206BEC3E8947FE994005028
:1006AF00030206BE787F79000206BE788079FF8844
:1006BF004A894B22E54A2547F8E54B3548F9854BE2
:1006CF0020E4300701F43549FA30E709C3EA94F022
:1006DF0040150206FCC3EA940F50030206FC78FF94
:1006EF0079FF7A0F0206FC780079007AF0C3E524CF
:1006FF009564500AC374019524500B02071AE54BF9
:10070F0020E70E02071AE54B30E706884789488A2B
:10071F00492278A4E6FAC3E54A33F8E54B33F9D119
:10072F002FE930E70BC3E89480E994FF4013E154BD
:10073F00C3E8947FE994005002E154787F7900E197
:10074F0054788079FFE820E715C3E52398F840092E
:10075F00C3E89401400302077B780102077BE8F4AA
:10076F0024012523F8400302077B78FF884C227869
:10077F00A5E6FAA848A949D12FE930E70CC3E894B8
:10078F0001E994FF40160207AFC3E894FFE9940014
:10079F0050030207AF78FF79000207AF780179FFA6
:1007AF00E920E715C3E54C98F84009C3E8940140E8
:1007BF00030207D678010207D6E8F42401254CF886
:1007CF0040030207D678FF88242278FFC26420698D
:1007DF003D206A12D264C3E541940A4009C3E5255E
:1007EF0094405002C26479A1E76023E541601F7411
:1007FF00FF8541F0848539F0306A0375F005A4F860
:10080F00C5F0600278FFC3E895675002A867886655
:10081F0022C3E5409440E5419401E566500314017D
:10082F0031046002F566220208392275E8902278B9
:10083F0083E6FFE5E820ECF7A8BDA9BE0573C3E585
:10084F007394084052757300E9FA79A0E76044EA9F
:10085F007007E574601B020874C3E895746010E5B7
:0F086F00745006600C140208800460F9020880BF
:10087E00E574F574C3946D401B7564C0C394044055
:10088E0013756480C39404400B756440C394044094
:10089E000375640075BB0622E564F460020564E529
:1008AE0073B4070375BB1022743279A687F0A4C502
:1008BE00F0A2F733F8C3E895644002A86488228852
:1008CE0024882588268867227540007541F022C24B
:1008DE00AF75C820A8CCA9CDAA3A30CF010A75C8E9
:1008EE0024D2AFAB3BAC3C883B893CC3E89BF8E9D8
:1008FE009C206908F930670221F2214FAD3D8A3DF7
:10090E00F9EA9DFA600478FF79FFAE3EAF3F8B3E69
:10091E008C3FC3EC9FFCC3E99CF542A83BA93CC3AA
:10092E00E89EF8E99FF9C3E54113FBE54013FAE8A9
:10093E002AF540E93BF54150067540FF7541FF2110
:10094E0099AA40AB41AC40AD417E047F02C3EB940B
:10095E000440021E1FC3EB940840021E1FC3ED137A
:10096E00FDEC13FCDEF7C3EA9CFAEB9DFBEF60098E
:10097E00C3E913F9E813F8DFF7EA28FAEB39FB8A33
:10098E00408B4150067BFF8B408B41C3EB94025052
:10099E0002D2673069047F0321C47892E6FFC3E573
:1009AE0037948240110FC3E53794A040010FC3EF77
:1009BE00940640027F057E04E541C4540FF9E541DB
:1009CE00C454F0F8E540C4540F28F8C3E89EFAE981
:1009DE009400FB4009C3EA9402EB940050047A029F
:1009EE00E4FB413EAA40AB41EBC4FEEAC4540F4EB9
:1009FE00FCC3EA9CFAEB9400FBC3E813C313F8EABA
:100A0E0028FAEB3400FB8A408B41C3EB9402400280
:100A1E00C2677804EBC4FE7B00EAC4540F4EFAC3DF
:100A2E00EA98FA4005C3940250027A027892E6FFE1
:100A3E00306002413E855256855357D26043E68060
:100A4E00C3E49AF8E49BF930670241D8E8FAE9FB6F
:100A5E00D3E913FDE813FC88528953C3EF94036066
:100A6E0038EF20E00DE82CF8E93DF9ECFAEDFB0249
:100A7E000A93E828F8E939F9C3E82402F8E93400C2
:100A8E00F97AFE7BFFC3EF9403400E8A548B558890
:100A9E004E894F8C508D51610C885489558A4E8BDE
:100AAE004F8C508D51306920C3E53394034019E5C6
:100ABE0042A2E713F8E555F4240138400B20E7086D
:100ACE007554FFF42401F555610CE8FAD3E813FCD4
:100ADE008852C3EF94036020EF20E007E82CF8EC77
:100AEE00FA41F8E8282402F87AFEC3EF940340088E
:100AFE008A54884E8C50610C88548A4E8C50E56B0B
:100B0E00C3335002646BF56B3060026116753402AC
:100B1E00D26043E680E52D54066026A840A941C365
:100B2E00E913F9E813F8C2AF53E67F759100C3E4F9
:100B3E0098F594E499F595759104D26043E680D2C8
:100B4E00AF22D265754400752000306B03752040CE
:100B5E00020B6FD265754400752040306B03752013
:100B6E0000D2AF7801206722E52D54066002C265DF
:100B7E00C3E5419405401378029405400878039428
:100B8E000540027806306902780A206019E5446053
:100B9E001530690AC3E53394034003D53406D2AF4A
:100BAE00D26C8140711ED2AF0000C2AF206726E525
:100BBE0041C3FB940F40027B0FEB240530730123DE
:100BCE00306A02742820620123F93069027982E5C5
:100BDE008BC39940B50544E59B5440B52002812A4C
:100BEE0030690A08C3E8940A40010861982065023A
:100BFE00616FC26553E67F75910030671075940082
:100C0E007595FE759104D26043E680616FAE40AF7C
:100C1E0041C3E49EF594E49FF5958111C3E53394A9
:100C2E00025002616F306502616FD802813E619899
:100C3E00C26C53E67F7591008554948555957591D8
:100C4E0004854E56854F57D26043E680D2AFE52DD0
:100C5E0054066008206A020533020C7A306C0D20AF
:0F0C6E006B0A206507158115810214F1227800A9
:100C7D003064053065027801E53775F007A4F9E5B4
:100C8D00F028F5F0E9A2F013A2F113A2F213F53753
:100C9D00C394785003753778C3E53795384008D23B
:100CAD0066C295C294C29330600281B48550568558
:100CBD005157D26043E68022207D11C2AF754302A9
:100CCD00D291C292D2AF759F11020E94C2AF7543ED
:100CDD0002D291C290D2AF759F11020E9430724321
:100CED00207D20C2AF75430390013C757E02C293F7
:100CFD00D290306204D294A108C291D2AF759F01F7
:100D0D00020E94C2AF75430390013C757E02C295ED
:100D1D00D292306204D294A128C291D2AF759F2194
:100D2D00020E94207D17C2AF754303900117C29335
:100D3D00306202D294D2AF759F01020E94C2AF758C
:100D4D004303900117C295306202D294D2AF759FC2
:100D5D0021020E94207D11C2AF754304D292C29030
:100D6D00D2AF759F21020E94C2AF754304D290C2CB
:100D7D0092D2AF759F01020E94307243207D20C236
:100D8D00AF75430590012B757E04C294D2913062EC
:100D9D0004D295A1A4C292D2AF759F11020E94C236
:100DAD00AF75430590014D757E01C294D2913062AD
:100DBD0004D293A1C4C290D2AF759F11020E94209C
:100DCD007D17C2AF75430590010DC294306202D2FA
:100DDD0095D2AF759F11020E94C2AF754305900168
:100DED0021C2943062EBD293D2AF759F11020E9453
:100DFD00207D11C2AF754306D290C291D2AF759FBF
:100E0D0001020E94C2AF754306D292C291D2AF7554
:100E1D009F21020E94307242207D20C2AF75430196
:100E2D0090014D757E01C295D292306204D293C16C
:100E3D0040C290D2AF759F21020E94C2AF7543018F
:100E4D0090012B757E04C293D290306204D295C16D
:100E5D0060C292D2AF759F01C194207D16C2AF754D
:100E6D004301900121C295306202D293D2AF759F9A
:100E7D0021C194C2AF75430190010DC2933062023E
:100E8D00D295D2AF759F01C2662290010B757E007F
:100E9D00C295C294C293D292D291D290C26222785C
:100EAD008076FF0876FF0876FF0876FF0876030840
:100EBD00760408760A087601087601087601788CA2
:100ECD0076010876FF0876FF0876FF0876FF08762C
:100EDD00FF0876030876FF0876FF0876FF0876256B
:100EED000876D00876FA0876FA0876040876FF08B0
:100EFD00760108760008767A0876FF08760108767E
:100F0D0001087600087603227887E6FFC27278889A
:100F1D00E6C394036008C27DE630E102D27DC27E55
:100F2D007889E630E102D27EC3EF94026008758EB7
:100F3D0001D273020F48758E00C273227880E614B9
:100F4D009000809378A4F67881E6149000809378D1
:100F5D00A5F67886E61490008D9378A6F6789CE633
:100F6D007538FF75390CB402067538A075390AB499
:100F7D00030675388275390578A3E61490009A93A7
:100F8D00F569D19722227896E6FA7897E6FB78886C
:100F9D00E6B40305C3EB940EFB307F047A007BFFB0
:100FAD00C3EB9AFCC3948250027C82757500057563
:100FBD00EC8575F0A4C3E5F0947D40F222D27FF16B
:100FCD009312058C7A007B007C10120582E55F2A56
:100FDD00FA74003BFBDCF37C04C3EB13FBEA13FA5E
:100FED00DCF7FEC27FF19322E5EF20E603752000CA
:100FFD000520903FFFE520146006901DFF14600052
:10100D009304600375EF1253D9BF7581C043FF8000
:10101D0012057D75EF0243B203E5B3240420E70DFD
:10102D00F521E5E320E0068521B343E301120E9798
:10103D007580FF75A40075F19075D47F75908775D7
:10104D00A5BF75F2BF75D50075A60175E241E4F82F
:10105D00F6D8FD756B01120EAC12153378988676A5
:0E106D00753001C2AF1205961205A612058C51
:10107B001205AD12058C1205B412058C12164C120A
:10108B000596120596120591C2AF78FA79FA308758
:10109B0007D9FBD8F7021C00120F15120F49120FBC
:1010AB0092120F9378988676120E977588507589E1
:1010BB001275C82475910475D84075A82275B802AD
:1010CB0075E690759B80759D0075D10E75BC587536
:1010DB00BB0675BA1175E88012057DD2AF120836C2
:1010EB0053DACF207E0343DA20307E0343DA1043FA
:1010FB00DA01C2D8C271120596D2617B037A0CE574
:10110B005E70077A0CDB0302109312058C207003C0
:10111B00021093C270E55FC3940240E1E52F541FA8
:10112B00856160F561B560D5DAD5C26153DACF2040
:10113B007E0343DA20307E0343DA10C2D8C27178C3
:10114B00A2E67008D274E52F54E0F52FC27575290D
:10115B0000120591307409C3E529940A4002D27537
:10116B0012058278023074027800C3E55F9840F074
:10117B00C2AF1205A61205A61205A6D2AF1205968E
:10118B00754D007888E6B403024173120582788CA2
:10119B00E6C394015003021273E530C3940150036C
:1011AB00021273207435C3E55F94FF500302127370
:1011BB00C2AF1205BBD2AF120591C3E55F940150CC
:1011CB00EFC2AF1205A61205871205A6D2AF120504
:1011DB0091C3E55F94FF40E90216D17F05D27F12E0
:1011EB000F93120591C2AFC27F120F93AE5FC3E58F
:1011FB005F947FD2AF407B12057DC2AF1205BBD28D
:10120B00AFDFDA120FCAC3EE94057897F612059684
:10121B001215751216547F0AD27F120F9312059175
:10122B00C2AFC27F120F93AE5FC3E55F947FD2AFA5
:10123B0050E412057DC2AF1205A61205871205A652
:10124B00D2AFDFD4120FCAEE24057896F6120596AC
:10125B00121575121683120591120F93C3E55F9445
:10126B00FF500221AE0216D1C3E55F954D400385B9
:10127B005F4D12059178017988E7B403027805C3B5
:10128B00E55F984002218EC2AF1205BB1205BB125F
:10129B0005BBD2AF120596753000E4F531F532057A
:1012AB0031E531F470390532789AE6781914601209
:1012BB00783214600D787D14600878FA1460037529
:1012CB003200C3E53298401715327531B4789986E0
:1012DB0076C2AF1205BBD2AF789886761205911203
:1012EB000587E52A7005307402019378012074029A
:1012FB007806C3E55F9840A77888E6C3940360033C
:10130B00120591E52A7003021093C2AF120E97E4F7
:10131B00F522F523F524F525F526F56AD2AF788568
:10132B00E6C333F568E4F545F546F547F548F54969
:10133B00F573F52CF52DF53775730875BB10120584
:10134B007D12083AE5E820ECFBA8BDA9BEE97001C7
:10135B00F8887412083E75730875BB107887E6FE23
:10136B007602120F157887EEF6C2AF7564FF12087E
:10137B00B6852264852265852266D2AF75220175FA
:10138B00240175250175260185636C756D017888BF
:10139B00E6B40307C27D307602D27DD268D269757E
:1013AB003300120DFD120E221208D61208DD1208A0
:1013BB00D61208DD1208D60213D2C2AF120F15D205
:1013CB00AF75730075BB06120B61120686120C7B90
:1013DB00120CC51208DD120B50306D03120687205C
:1013EB0067031207D9306703120820120C7B120C0B
:1013FB00EA1208DD120B61306D031206C3120C7B6F
:10140B00120D611208DD120B50306D031207211201
:10141B000C7B120D861208DD120B61306D03120767
:10142B007E120C7B120DFD1208DD12083A120B50C6
:10143B00120C7B120E2212083E1208DD306932208C
:10144B006B2F85676485676585636C756D0179188E
:10145B007A0CC3E53399400CC269D26A8A3575643C
:0E146B00FF02147CC3E55F940140030213D21C
:101479000214F9306A1B206B18E535147004C26A2E
:1014890061C5F535C3E55F940140030213D2021427
:10149900F9753600C3E5627882985054307404E5D2
:1014A9002A604D7888E6B40317207D0520760781E8
:1014B900C930760281C9206B07D26B8567648111B7
:1014C90078F0306B058567647820C3E54198500250
:1014D90061D2306B1BC26BC27D307602D27DD26A7B
:1014E90075351285676461D20536E55F600281FC56
:1014F900753600C2AF120E977887E6FE7602120F94
:10150900157887EEF6E4F522F523F524F525F52679
:10151900F568C268D2AF12057D120E97307409C3FF
:10152900E53694054002019341A5901A0D782012E1
:1015390015B7E520B45A0CA31215B7E520B4A503D5
:10154900021555120EAC121575021574901A03780E
:10155900807B0A1215B7A308DBF9901A0F788C7BE8
:10156900181215B7A308DBF9901A2722C2AF121572
:10157900F61215D0901A00740E1215BCA374041239
:1015890015BCA374141215BC901A0378807B0A1237
:1015990015BBA308DBF9901A0F788C7B181215BBC1
:1015A900A308DBF91216091215E7901A2722E4930A
:1015B900F622E6438F01538FFD75EF0275B7A575C6
:1015C900B7F1F0538FFE22438F02438F0175EF026B
:1015D90075B7A575B7F1901A0DF0538FFC22901AC3
:1015E9000D745AB1BC901A0E74A5B1BC227A307927
:1015F900D07820901A40B1B7E520F709A3DAF7228D
:101609007A3079D0901A40E7B1BC09A3DAF922AB54
:1016190077A878BB01027984BB02027985BB0302F2
:101629007986BB04027992BB05027987BB060279E8
:10163900A3BB0702799CBB08027988BB0902798997
:10164900E8F7227C05120596DCFB22C2AF1205A63B
:101659001205AD1205B41205BB1205871205A612B3
:1016690005AD1205B41205BB1205871205A61205B0
:10167900AD1205B41205BBD2AF22C2AF1205BB121F
:1016890005B41205AD1205A61205871205BB120590
:10169900B41205AD1205A61205871205BB1205B4D1
:1016A9001205AD1205A6D2AF22AE77AF78C2AF123E
:1016B90005A61205A61205A6120587DEF21205BBBC
:1016C900120587DFF8D2AF22D154D14CD14C7577AE
:1016D90001757801757900D1B27C05AD5F12059667
:1016E900C3ED955F70F5C3E55F9401400AC3E55FFB
:1016F90094FF403202170DD118B175D154C2AF759C
:10170900EF12D14CDCD50579C3E5799403500280F9
:10171900C6D14C0578E5771490009F93F808C3E586
:101729007898500280AED14CD14C0577C3E57794B7
:101739000A5002809C120EACB175C2AF75EF12D17E
:011749004C53
:0319FD00020FF5E1
:101A00000E0414FFFFFFFF03040A0101015AA501A0
:101A1000FFFFFFFFFF03FFFFFF25D0FAFA04FF01DE
:081A2000007AFF01010003FF41
:101A400023585031384123202020202020202020DE
:101A500023424C48454C4923463333302320202031
:101A60002020202020202020202020202020202076
:101C0000C2AFC2D353D9BF7581C043B20343FF8073
:101C1000752438752503B1C975EF0275E24043F1AB
:101C20008053A47F75D400D2877DFA780379E67C4F
:101C300010752200752300901DD67B0675249875BB
:101C400025013087028142208708D8FBD9F9DCF7CB
:101C500081B4308708D8FBD9F9DCF781B4B189E4C5
:101C600093A3C39A6004DDC381B4DBDBB17B600264
:101C7000812B7B08E493FAA3B15CDBF87A30B15C8A
:101C8000752200752300B17BEAFCEBFDC3ED94FEE9
:101C9000400EB17B8A278B28ED30E0048A828B834B
:101CA000B17B7AC270D8C3ED94FE601350CEBD00F4
:101CB00025EC60097520007521FF0200008100A855
:101CC00027A9280809D804D90281D3B17FEA89AAB3
:101CD000F281C50D81A0C3ED94035049EDA2E092BD
:101CE000007AC5C3E5829400E583941C50902000DF
:101CF00010438F02438F0175B7A575B7F1F030001F
:101D00001FA827A9280809438F01538FFDD804D99C
:101D100002A12089AAE275B7A575B7F1F0A3A10DBC
:101D2000538FFC817C7AC1BD030CE493A3FAB140CC
:101D3000DCF8B138817C817EAA22AB23B15CEBFA5E
:101D4000EA6222752608C3E52313F523E52213F57D
:101D50002250066323A0632201D526EAB1C9B1C986
:101D600075260AEAF4200102D287300102C287B147
:101D7000C9C3134002C201D526EB22B17FEAFB2082
:101D80008702A17F308702A184752608AE24AF2583
:101D9000C3EF13FFEE13FEB1CDB1C9C3EA13308711
:101DA000024480FA30E703632201C3E52313F523DD
:101DB000E52213F52250066323A0632201D526D91C
:101DC000E52265236523F52222AE24AF250E0FDE22
:101DD000FEDFFCD20122424C48656C693437316326
:041DE000F3300601D5
:00000001FF
